:020000040000FA
:060000000C3003303A2829
:08000800A000030EA100831209
:1000100005191028831601178312B23081002B288E
:1000200083160113831203140B190310A80DA90DD5
:10003000AA0DAB0DAC0DAC16FF302C02031D2B2806
:10004000FA302B02031D2B2831152A08AF0029088E
:10005000AE002808AD008B100B11210E8300A00EFE
:04006000200E090065
:0C007400203084008001840A6030040207
:10008000031C3C281230B00075218316FF2390001A
:10009000831283160C308505870183128501870141
:1000A000073099000030831691009F008312C830FA
:1000B00083168100831231309000003083168C004B
:1000C000831210308B00BB2181018E018F010B1137
:1000D0008B100B108C018B1791217D203119802002
:1000E0005921B30B7B28031085190314B90DF03087
:1000F00039020319F520C0216D2864003210080070
:1001000031110130B7008B132030370783169B0065
:100110001C141A088312A4001030370783169B00A2
:100120001C141A088312A300A6000230A606003091
:10013000370783169B001C141A088312A200A7001D
:100140000130A7068B17321CAB2822090339A20005
:10015000A309A409A50924082F02031DEF282308D9
:100160002E02031DCA2822082D02031DEF2801308C
:100170003702031DC128C0283D18C1283D143E1474
:10018000912102303702031DCA28BD18CA28BD14A8
:100190003E14992126082E02031DE62827082D0269
:1001A000031DEF2801303702031DDC28DB283D1C2E
:1001B000DC283D103E149C2102303702031DE52847
:1001C000BD1CE528BD103E14A421EF285F08F039BE
:1001D000A03C0319EF282E1AEF28EE28A721B70A12
:1001E000033037020318080083280130B600B3003B
:1001F000B400B500B70085018701B113B4217D209B
:10020000B30B2729031085190314B90DF0303902F7
:1002100003194E29B41F8501B41F8701B40B272988
:100220000230370203191829B50B27290230B5000F
:10023000013037020319AA21023037020319AF2116
:10024000FA30B4000230370296300319B400311D81
:10025000FF283111321C31292D090339AD00AE09B7
:10026000AF092F1CFF288E018F010C1CFF280C10DA
:100270002E1EFF288B1320303707BB002F08BA0033
:10028000622110303707BB002E08BA00622100300F
:100290003707BB002D08BA0062218B17B7218501F3
:1002A0008701B70AB60103303702031CFF28BB21C0
:1002B00008003E1C08003E101030BB003D08BA008C
:1002C000622108008B133A0883161C159A003B081C
:1002D0009B0055309D00AA309D009C1464009C1822
:1002E0006E291C1183128B170800831600309B00A7
:1002F0001C141A088312DF00831610309B001C1494
:100300001A088312BD00831620309B001C141A08A3
:100310008312C1000130C11BC100C1080319C10013
:100320000800051205148E018F010C104108C00051
:100330000800851285140800051005168E018F012E
:100340000C104108C0000800851685100800051033
:1003500005120800380911398500B800080038096D
:1003600022398500B8000800B80138140800B80127
:10037000B814B8160800BD188514BD1C85160800F1
:100380005F080F390A3C0319CE290C1C6D280C108C
:0E039000C00B6D284108C000051005120800C2
:084000000A000300050008009E
:02400E00CC01E3
:10420000010078007A007C007E007B0079007F004E
:104210007D007A0078007E007C00FF00FF00FF0038
:104220000000F200F600FA00FE00F200F600FA00CC
:10423000FE00F200F600FA00FE00FF00FF00FF00A3
:10424000010005000500050005000900090009003E
:1042500009000D000D000D000D00FF00FF00FF0024
:10426000FF00FF00FF00FF00FF00FF00FF00FF0056
:10427000FF00FF00FF00FF00FF00FF00FF00FF0046
:10428000FF00FF00FF00FF00FF00FF00FF00FF0036
:10429000FF00FF00FF00FF00FF00FF00FF00FF0026
:1042A000FF00FF00FF00FF00FF00FF00FF00FF0016
:1042B000FF00FF00FF00FF00FF00FF00FF00FF0006
:1042C000FF00FF00FF00FF00FF00FF00FF00FF00F6
:1042D000FF00FF00FF00FF00FF00FF00FF00FF00E6
:1042E000FF00FF00FF00FF00FF00FF00FF00FF00D6
:1042F000FF00FF00FF00FF00FF00FF00FF00DD00E8
:00000001FF
